:1000000008308A00002800005436E135EF366539A3
:10001000203765316F10F63CF335EF366539A006B1
:100020000A00D43270366F3A611DA01231182E1AB0
:100030006614733A7538EE32A9060A005436E13573
:100040003A10A518301734332828E1140D050001A3
:100050005634FD349A346B3461343A3420342534C8
:10006000313430342E343434663428346D34293409
:100070000D340A3400348316861183128611083039
:10008000F80042280000F8175328F813BA0C031898
:100090008615031C8611781753287813F80B462809
:1000A0005128000086153F308400840B552800003D
:1000B000F81B4528781B4D280800831603178C175A
:1000C0000C140000000083120C087F390319A128CA
:1000D0000313AD0003170D080313AE0003170F0839
:1000E0000313AF002D08BA003B202E0803178D0024
:1000F00003132F0803178F0083168C170C140000AE
:10010000000083120C0D0E0D7F390319A128031373
:10011000AD0003170D080313AE0003170F080313F8
:10012000AF002D08BA003B202E0803178D000313E3
:100130002F0803178F008D0A03198F0A03135D28F8
:10014000031703138A150A1221280830F80000004B
:1001500086108316861000008312BE0D0610031C45
:10016000B4288316061483120318B92883160610C0
:100170008312831686148312861CBC28F80BA728CA
:100180000000861083168610000006140000000090
:1001900086148312861CCA28F801000006187814F9
:1001A000861083168610831206108316061083129B
:1001B000080083160614000086140000831206103F
:1001C0008316061000008312861083168610C03036
:1001D0008312BE00A5202630BE00A520B830BE0088
:1001E000A52083160610000086148312861CF628AC
:1001F0000000FA2800008316061400000614000010
:100200008614000083120610831606100000831265
:10021000861083168610C0308312BE00A5201330CE
:10022000BE00A5200730BE00A520831606100000E2
:1002300086148312861C1A2900001E2900008316CA
:100240000614000006140000861400008312061035
:100250008316061000008312861083168610C030A5
:100260008312BE00A5202630BE00A5203930BE0076
:10027000A52083160610000086148312861C3E29D2
:1002800000004229000083160614000083128A151C
:100290000A1224282E3084008313000803195D29D4
:1002A0000230F800F701F70B5329F80B5229973069
:1002B000F700F70B5929800B502908008316061404
:1002C000000086140000831206108316061000003A
:1002D0008312861083168610C0308312BE00A520BC
:1002E0003C08BE00A52083160614000086140000FA
:1002F0008312861C792906108316061000008312CB
:10030000861083168610C1308312BE00A520F70127
:100310000830BF007708C00083160614000086145A
:100320008312861C912906180314061C0310F80D6D
:1003300000008316861083128610BF0B8C2983164B
:10034000061400008312061040080319AA29831618
:10035000061083120000831686148312861CAE29B1
:100360000000861083168610000083120610831684
:10037000061078088312BD0083160610000086144C
:100380008312861CC1290000C529000083160614AB
:10039000000083123D08F80008008E30F7003E0888
:1003A000F8003D08F900FA01F808031DE129790871
:1003B000F800F9010830F702F808031DE129F701F8
:1003C000E9290310F81BE829F90DF80DF703E129D5
:1003D000F813080041080319AF2ACD004508031996
:1003E000AF2ACD02031CF9297F30CD070318AF2AAD
:1003F000FF298130CD02031CAF2A0319AF2A4D0813
:10040000F700F801F901FA01CC014208CB00CB1743
:100410004308CA004408C9001930CD004808C90281
:100420000318222A0130CA020318222ACB02031819
:10043000222ACC020318222ACC0ACB0ACA0A48086C
:10044000C907542A4708CA0203183D2A0130CB02C3
:1004500003183D2ACC0203183D2ACC0ACB0A4708D0
:10046000CA074808C907031C542ACA0A031D542A8C
:10047000CB0A031D542ACC0A542A46088038CB02E2
:100480000318532A0130CC020318532ACC0A460819
:100490008038CB074708CA07031C312ACB0A031D43
:1004A000312ACC0A312A7A14CD0B572A622A03103A
:1004B000C90DCA0DCB0DCC0D0310FA0DF90DF80DB9
:1004C000CE0D0E2A4E1C6A2A0310F80CF90CFA0CF9
:1004D000CE0C6D2AF7030319AF2ACE1B962A031000
:1004E000C90DCA0DCB0DCC0D4808C9020318822ACC
:1004F0000130CA020318822ACB020318822ACC02D6
:10050000031CA52A4708CA0203188D2A0130CB0212
:1005100003188D2ACC02031CA52A46088038CB027A
:100520000318962A0130CC02031CA52AFA0A031DDF
:10053000A52AF90A031DA52AF80A031DA52AF70A08
:100540000319AF2AF80CF90CFA0C4208CD00460842
:10055000CD06CD1FAD2AF817B32AF813B32AF70139
:10056000F801F901FA01080080308318C806CD01AE
:10057000CE014408CC004808CC0643080319A42B3C
:10058000CB00F70047080319AD2BCB020319492B09
:10059000031C072B4808D100D1174908D0004A088E
:1005A000CF00CE010310D10CD00CCF0CCE0CCB0B56
:1005B000D12ACC1FDE2A4D14C12B4D104B104D16E5
:1005C000463084008313D62B4D12CC1BF12A4B1CD2
:1005D000FC2AD10CD00CCF0CCE0CF70A0319BC2B83
:1005E000FC2AD11BFF2A0310CE0DCF0DD00DD10D4B
:1005F000F7030319BC2BF12A4D17692B4D1344083F
:10060000CC00CC1F052BD117B52BD113B52B470828
:10061000CB00F7004308CB024408D100D1174508AE
:10062000D0004608CF00CE010310D10CD00CCF0C67
:10063000CE0CCB0B132BCC1F202BCD14C12BCD10EC
:100640004B10CD164A3084008313D62BCD12CC1B11
:10065000332B4B1C3E2BD10CD00CCF0CCE0CF70AFD
:100660000319BC2B3E2BD11B412B0310CE0DCF0DFC
:10067000D00DD10DF7030319BC2B332BCD17692BEC
:10068000CD134808CC00CC1F472BD117B52BD11365
:10069000B52B4808D100D1174908D0004A08CF002F
:1006A000CC1F562BD1134D15C12B4D11CE014B1024
:1006B000463084008313D62BCC1B7F2B4408CC0000
:1006C0004B1C692BD10CD00CCF0CCE0CF70A0319A4
:1006D000BC2BCE1F7A2BCF0A031D7A2BD00A031D09
:1006E0007A2BD10A031D7A2BD10CD00CCF0CF70A30
:1006F0000319BC2B4D1BFE2ACD1B402B9E2B80309B
:10070000D106D11F872BC12B4808CC00942B44085D
:10071000CC00D108031D942BD008031D942BCF08C7
:10072000031D942BF701B52BD11B9E2B0310CE0D6F
:10073000CF0DD00DD10DF70B942BBC2BCC1FA22BC2
:10074000D117B52BD113B52B4708F7004808D100B6
:100750004908D0004A08CF00B52B4308F7004408E9
:10076000D1004508D0004608CF005108F8005008D5
:10077000F9004F08FA00F42BF701F801F901FA012A
:10078000F42BCE01CF09D009D109CE09CE0A031D21
:10079000CF2BCF0A031DCF2BD00A0319D10A4D1836
:1007A000DD2ACD181F2B4D19552B842B0008CF07A0
:1007B000031CE02BD00A031DE02BD10A03194B14B4
:1007C00084030008D007031CE82BD10A03194B143B
:1007D00084030008801F803AD10703184B144D1A78
:1007E000E42ACD1A262B5C2B08000430BC005E21C5
:1007F0007808AD000530BC005E21780EF7000F30A0
:10080000F7057708BE01BD00CD217708B60078084E
:10081000B7007908B8007A08B900C4007908C300A5
:100820007808C2007708C100C801C701C60183303B
:10083000C500EA217A08B1007908B0007808AF0055
:100840007708AE00BE012D08BD00CD2183107A08C7
:10085000C6007908C5007808C4007708C3003108CD
:10086000CA003008C9002F08C8002E08C700B422EB
:100870007A08B5007908B4007808B3007708B200A8
:100880003208F7003308F8003408F9003508FA0098
:100890008A150A1230280130BC005E21B001AF0178
:1008A000AE017808AD000230BC005E21B2017808CC
:1008B000B1000330BC005E217808B300330EF700AE
:1008C0000F30F7057708BE01BD00CD217708BD00C8
:1008D0007808BE007908BF007A08C000C400790813
:1008E000C3007808C2007708C100C801C701C6016B
:1008F0008130C500EA217A08BB007908BA0078087F
:10090000B9007708B800BD012D0DBE002E0DBF0047
:100910002F0DC000BE0DBF0DC00DFC30BE05310D4A
:10092000F900320DFA00F90DFA0DFC30F9057908DD
:10093000BD047A08BE04330EF700F70CF70C033041
:10094000F70577083D04F7003E08F8003F08F90076
:100950004008FA007A08C6007908C5007808C40083
:100960007708C300B630F700FA01F901F80143082F
:10097000440445044604031DBF2CF701CC2C03108E
:10098000F81BCB2CC30DC40DC50DC60DFA0DF90D0A
:10099000F80DF70BBF2CF8137708BD007808BE00E0
:1009A0007908BF007A08C00083107A08C600790869
:1009B000C5007808C4007708C3003B08CA003A089D
:1009C000C9003908C8003808C700B4227A08B7003F
:1009D0007908B6007808B5007708B4003408F70045
:1009E0003508F8003608F9003708FA008A150A12A7
:1009F0003B2883160614000086140000831206109C
:100A00008316061000008312861083168610C030ED
:100A10008312BE00A5202630BE00A520B830BE003F
:100A2000A52083160610000086148312861C162D3E
:100A300000001A2D000083160614000006140000A2
:100A4000861400008312061083160610000083121D
:100A5000861083168610C0308312BE00A520133086
:100A6000BE00A5200730BE00A5208316061000009A
:100A700086148312861C3A2D00003E2D000083163A
:100A800006140000061400008614000083120610ED
:100A90008316061000008312861083168610C0305D
:100AA0008312BE00A5202630BE00A520B930BE00AE
:100AB000A52083160610000086148312861C5E2D66
:100AC0000000622D000083160614000083128A15B0
:100AD0000A1246280130BC005E21AE017808AD0044
:100AE0000230BC005E217808AF000330BC005E21FC
:100AF000780EF7000F30F7057708BE01BD00CD2155
:100B00007708B8007808B9007908BA007A08BB00FD
:100B1000C4007908C3007808C2007708C100C80182
:100B2000C701C6018330C500EA217A08B3007908FD
:100B3000B2007808B1007708B0002D08BA00B901FA
:100B400039082F04F7002D08FA007708BD002D089A
:100B5000BE00CD217708B9007808BA007908BB003B
:100B60007A08BC0083107A08C6007908C5007808A6
:100B7000C4007708C3003308CA003208C90031082E
:100B8000C8003008C700B4227A08B7007908B60058
:100B90007808B5007708B4003408F7003508F80085
:100BA0003608F9003708FA008A150A125228831607
:100BB00003178C170C14000000000318062E831274
:100BC0000C087F390313AE0003170D080313AF00A1
:100BD00003170F080313B0002E08BA003B202F089C
:100BE00003178D000313300803178F0083168C172B
:100BF0000C140000000083120313AD0B002E032E13
:100C000083160317062E252E8316031783120C0D49
:100C10000E0D7F390313AE0003170D080313AF0049
:100C200003170F080313B0002E08BA003B202F084B
:100C300003178D000313300803178F008D0A031963
:100C40008F0A03100313AD0BD72D0800F701F8012D
:100C5000F901FA01C201C301C401C5014108400400
:100C60003F043E040319642E2030C6000310BA0D61
:100C7000BB0DBC0DBD0DC20DC30DC40DC50D41088E
:100C80004502031D4D2E40084402031D4D2E3F0812
:100C90004302031D4D2E3E084202031C5E2E3E08F9
:100CA000C2023F08031C3F0FC3024008031C400F51
:100CB000C4024108031C410FC5020314F70DF80DCF
:100CC000F90DFA0DC60B362E42308400831308004E
:100CD0000408B2003108B4000319FA2E3008BD0030
:100CE0002F08BC002E08BB002D08BA00C101C001AE
:100CF0002030BF008230BE003A080319EC2EC2003B
:100D00003E080319EC2EC20703188D2E7F30C20255
:100D1000031CEC2E0319EC2E912E8130C207031810
:100D2000EC2E4208F700F801F901FA013B08C60071
:100D3000C6173C08C5003D08C4001830C200C301F6
:100D4000441CBA2E4108FA07031CAC2EF90A031DF5
:100D5000AC2EF80A0319C3174008F907031CB32E79
:100D6000F80A0319C3173F08BC00BC173C08F80772
:100D70000318C317C30DF80CF90CFA0CC60CC50CFC
:100D8000C40C0310C20B9F2E0130F7070318EC2E82
:100D9000F81BD12EC60DFA0DF90DF80DF703031946
:100DA000EC2EC61FE22EFA0A031DE22EF90A031DDD
:100DB000E22EF80A031DE22EF80CF90CFA0CF70AE1
:100DC0000319EC2E3B08C3003F08C306C31FEA2EDD
:100DD000F817F02EF813F02EF701F801F901FA01D7
:100DE0007A08B0007908AF007808AE007708AD0047
:100DF000B40B6E2E3008BD002F08BC002E08BB00BF
:100E00002D08BA003A08B63CBA00FA013B08BE0009
:100E1000BB170310BB0CBC0CBD0CFA0CF90CF80C86
:100E2000F70CBA0B092FBE1F202FF709F809F90993
:100E3000FA09F70A0319F80A0319F90A0319FA0A51
:100E40007A08B0007908AF007808AE007708AD00E6
:100E5000B01F372FB203B216AD09AE09AF09B00902
:100E6000AD0A0319AE0A0319AF0A0319B00A3B30E1
:100E7000B9009A30B800CA30B700B6010A30B400E1
:100E800031080319B20A3008BD002F08BC002E0833
:100E9000BB002D08BA003908C1003808C000370867
:100EA000BF003608BE0026260008AD00840A0008F0
:100EB000AE00840A0008AF00840A0008B000FD30CC
:100EC0008407F708031D772F310A34020319772F9F
:100ED00032080319792F0F3934020319712F0318BF
:100EE000A92FB21BA92F321B792F2030A52F20301C
:100EF000B205B21E872FB2123108031DB203770864
:100F0000B2002D30BA003B203208F700B2013108A0
:100F10003402031D952F7708B2002E30BA003B2013
:100F20003208F7002030B20500303030B21EA52F55
:100F3000B2123108031DB2037708B2002D30BA0097
:100F40003B203208F700B2013030F7077708BA00CB
:100F50003B203908BD003808BC003708BB00360804
:100F6000BA00C101C001BF010A30BE0026267A08BE
:100F7000B9007908B8007808B7007708B600B40B54
:100F8000432F0800831603178C170C140000000071
:100F900083120D080313AE0003170F080313AF00ED
:100FA00003170C080313BA003B202E0803178D000B
:100FB00003132F0803178F008D0A03198F0A0313D9
:060FC000AD0BC22F08007A
:10100000840183131F308305713083168F000F080E
:10101000861183128615831603170908C0398900C3
:1010200003131F129F1200300317880083128701D9
:101030008801890104308D0000308F008A1103136C
:101040005D288A158A11D9288A150230AD00FA3038
:10105000AE008A114A218A15AD0B27288A11F52B7B
:101060008A157A08A8007908A7007808A6007708EA
:10107000A5008A114B2C8A157A08A4007908A300D0
:101080007808A2007708A1008A11F92C8A1502308D
:10109000AD00FA30AE008A114A218A15AD0B4928FD
:1010A0008A116A2D8A157A08AC007908AB00780895
:1010B000AA007708A900113003178D0000308F00B7
:1010C000031009300313AD008A11D7258A150930A2
:1010D00084002808B0002708AF002608AE002508C5
:1010E000AD000430B1008A1168268A151830031744
:1010F0008D0000308F0003140A300313AD008A11F5
:10110000D7258A151E3003178D0000308F0003107D
:1011100006300313AD008A11D7258A1509308400E3
:101120002408B0002308AF002208AE002108AD005B
:101130000430B1008A1168268A15243003178D0007
:1011400000308F00031006300313AD008A11D7253D
:101150008A15283003178D0000308F0007300313E5
:10116000AD008A11C2278A15093084002C08B0000E
:101170002B08AF002A08AE002908AD000430B100EA
:101180008A1168268A15353003178D0000308F00CC
:1011900005300313AD008A11C2278A150430AD0053
:1011A000FA30AE008A114A218A15AD0BD0282228C8
:0211B0006300DA
:04400E00F52CFF3F4F
:00000001FF
